:020000020000FC
:0E00000008ED04BF01E0009361000C94A6021D
:100400000C94A6020C9448020C9448020C944802E6
:100410000C949A020C9448020C9448020C94940296
:100420000C9448020C9448020C9448020C94480224
:100430000C9448020C948A020C9448020C944802D2
:100440000C9448020C9448020C9448020C94480204
:100450000C9485020C9448020C9450020C944802AF
:100460000C9448020C9448020C9448020C944802E4
:100470000C9448020C9449020C9448020C944802D3
:100480000C9448020C9448020C9448020C944802C4
:1004900018953090A9043092A904B599E69A189558
:1004A0002FB60F931F93EF93FF93009110061091B7
:1004B0001106F9E2EB2DEE0F01931193B394B2FE06
:1004C00002C0E49A14C003E0B01680F000E100938B
:1004D000A00000E00093010606E4009302060EE18E
:1004E0000093060601E00093080601C006D0FF91C4
:1004F000EF911F910F912FBE189504E00B0D009303
:10050000060601E0009308060895309069043092D1
:10051000690418953090960A3092960A2FB6550CB9
:10052000779B53942FBE189530900B0A30920B0A8C
:10053000E29A18952FB63090530130925301E79804
:10054000E69BE79AE69866242FBE189500E801B965
:1005500000E500B908E000931104009317040CE0D3
:100560000093100401E009B901E008B900E00DB9F9
:1005700000E00CB909E00093770404E000937404F0
:1005800000937504009376040CE0009370040093CC
:100590007104009372040093730408E005BB00E04B
:1005A00004BB01E00093B5040CE00093B204009397
:1005B000B60400E0009300060FE70093030608E08E
:1005C0000093050601E000930A0601E0009300068F
:1005D00008E01DE30093260A1093270A01E0009328
:1005E0000A0A0BE00093000A00E712E000938C0A6D
:1005F00010938D0A05E00093800A01EE14E0009349
:100600009C0A10939D0A01E00093950A05E000936F
:10061000900A01E00093470101E00093520100912C
:10062000510100FDFCCF01E700935001009101143E
:100630000395A1F40E945B0AE8E1F5E1A1E0B4E1D1
:10064000159101D00BC005910D931A95E1F71DE9A5
:1006500014BF13E0109300100C945B0A5524DD24A2
:10066000EE2400270CBB0DBB2DD031D005E000934C
:100670005000789411D0DE1029D5B499FCD2E09BBB
:100680004ED0E49998D2E59959D30799D4D0079BD5
:10069000E1D0E2992FD6EECF0FEF50120895002748
:1006A0000093500100270093B50421D0CED003E081
:1006B0000093A2044898889508ED04BF01E00093D8
:1006C000410008950091071402700DBB08951F9317
:1006D000AF93BF9300270EBB0FBB1EE3A8E0B9E2A8
:1006E0000D931A95E9F7BF91AF911F910895E09B83
:1006F000089500E20093E3050DE20093A60801E0EF
:100700000093A30801E00093A50814E021E070D055
:1007100014E022E06DD000270093A3087AC0519B1B
:100720000895B5D6B4D6B3D6E09AE09B089500E21A
:100730000093E3050DE20093A60801E00093A308EF
:1007400001E00093A50814E028E152D015E020E470
:100750004FD016E02FE94CD017E02FE749D018E032
:1007600020EF46D019E02FEF43D01AE020E040D030
:10077000C2EBD9E210E521E01DD019E521E01AD045
:1007800011E521E017D01091B2290091B3291C7016
:10079000007E110F02950695012B112726E731E007
:1007A000200F311F2093B2293093B32900270093E3
:1007B000A308089500E10093A70835D056F11093DF
:1007C000A80831D036F101E00093A40801E10093BC
:1007D000A70821D0F6F00091A80809932A9521F0E6
:1007E00002E00093A408F5CF07E00093A408089561
:1007F00000E10093A70817D066F01093A80813D063
:1008000046F02093A8080FD026F003E00093A40838
:100810000895E0985CCF2ED60091A50807FD0895B5
:1008200032D6D6F7089526D60091A50806FD08957C
:100830002AD6D6F70895519B08C0119B0E941F0528
:100840000E94AF050E941109089500270093C00877
:1008500007980895519B08950F9A079A00E2009314
:10086000C00800E30093C00804E00093C10801E35E
:100870000093C0080F9800EC0E94600A0F9A0E9433
:10088000470A1FEF0F9803E00E94600A0EE00E94E3
:10089000600A012F0E94600A0F9A007E003879F7E3
:1008A00011E00F9802E00E94600A08E20E94600ACC
:1008B000012F0E94600A0F9A1EE80F9802E00E9422
:1008C000600A09E20E94600A012F0E94600A0F9AE2
:1008D0001091181410640F9802E00E94600A0AE256
:1008E0000E94600A012F0E94600A0F9A50EF48E0B0
:1008F000309117142091161410E08CD030911B14F5
:1009000020911A1418E086D03FEF2FEF14E082D028
:1009100058EF442710E27ED014E27CD011E0009121
:10092000071404FD12600F9802E00E94600A0BE2B7
:100930000E94600A012F0E94600A0F9A10E00F982F
:1009400002E00E94600A0FE00E94600A012F0E94EC
:10095000600A0F9ACAE4D9E250EF48E030911714C8
:1009600020911614002718E059934993399329933D
:10097000099328961A95C1F749E0409358294BE00E
:100980004093652948E24093722948E440937F29C7
:1009900049E440938C294AE4409399294BE44093DD
:1009A000A6290F9802E40E94600A00EF0E94600AE4
:1009B00008E20E94600A00911B140E94600A0091E4
:1009C0001A140E94600A00270E94600A0F9A0F986A
:1009D00004E40E94600A01EF0E94600A09E00E949C
:1009E000600A00911B140E94600A00911A140E9470
:1009F000600A01E00E94600A009119140C700E94C4
:100A0000600A0F9A77240FE5802E9924AA240AE021
:100A1000C02E08950F9802E00E94600A012F0E94E4
:100A2000600A052F0E94600A042F0E94600A032FAB
:100A30000E94600A022F0E94600A0F9A08950F9880
:100A400000EA0E94600A0E94600A0F9A0F9300FD5C
:100A500004D00F9101FD4FD00895E69A0F9800E958
:100A60000E94600A0E94600A502F0E94600A402F74
:100A70000E94600A302F0E94600A202F0E94600AA4
:100A8000102F0E94600A002E0F9A43FF0895042F32
:100A9000569547954695469503704C7F402B1F70A1
:100AA000403079F0413081F0433089F0443091F0AA
:100AB0004F3099F04132D1F04232D1F04632D1F08C
:100AC0000895689490F80895689491F8089568944A
:100AD00093F80895689494F80895112321F0902CC8
:100AE000689497F808950BE9902E0895E89A089570
:100AF000E89808955CC30F9804E90E94600A0E9478
:100B0000600A502F0E94600A402F0E94600A302F16
:100B10000E94600A202F0E94600A102F0E94600A23
:100B20000E94600A0E94600A0E94600A0E94600A95
:100B3000002E0F9A43FF0895042F5695479546952A
:100B4000469503704C7F402B1F70443009F0089588
:100B5000153008F40895702C8824EC9A08950DE05F
:100B6000A09ECAE4D9E2C00DD11D1C811F70F9F00E
:100B7000FE011930D0F40F9800EA0E94600A0E942A
:100B8000600A0F9A02FD08950F9800E40E94600A1F
:100B90001B5F09910E94600A1A95D9F70F9A00000D
:100BA0000F9801E80E94600A0F9A11271483A394FA
:100BB000A3FCAA240895E49800910029109101292A
:100BC0002BE9129FA001029F0024410D501D40936C
:100BD0002A2950932B290091022910910329015EA3
:100BE0001E47409106145527EAEBF5E1E40FF51F87
:100BF00024911203A001029F0024410D501D24E006
:100C000052038001429F0024010D101D00932E29E4
:100C100010932F290091042910910529045119419D
:100C20002227332717FD890123EB129FA001029F82
:100C30000024410D501D27E0529F8001429F002457
:100C4000010D101D00932C2910932D2900910629C8
:100C50001091072920912111332727FD3FEF021B17
:100C6000130B209120111203A001029F410D41514D
:100C7000409326290895E09B089500E20093E30540
:100C80000DE20093A60801E00093A30801E00093A1
:100C9000A508C5EBD9E210E021E08CDD2A91A8DDA2
:100CA00027FF0895E19825FD12CDE19A1CE026E288
:100CB00081DD2091B2293091B3299FE0E091B429E0
:100CC000FF27E7FDFFEFA5EBB9E2C8E0D9E21D91F0
:100CD0000D918827029FA001139FB001039F500D23
:100CE000611D781F129F500D611D781F40505E4F8F
:100CF0006F4F7F4F76956795579576956795579582
:100D00005E0F6F1F599369939A9509F71296C7E280
:100D1000D9E204D003D002D0E59A08950D911D9137
:100D2000110F001F110F001F07FD0FE71127EAE346
:100D3000F5E1E00FF11F049109930895E59807D0BC
:100D400053D0C6D0DAD0EED057D168D108950090F4
:100D5000041410900514442755276FEF7FEFA8E087
:100D6000B9E2C4E3D9E2E3E4F9E215D014D013D038
:100D7000409330295093312960933229709333295D
:100D800088279927A4E3B9E222D021D020D08D93DF
:100D90009D939C0122C001E01127882799272D915E
:100DA0003D911694079458F4420F531F28173907A2
:100DB00010F0C901102F2617370708F4B901000FEA
:100DC00005FFEDCF899399932196119308952D9165
:100DD0003D912817390708F0C901261B370B00275A
:100DE00030132FEF2D930895A7E2B9E2C4E3D9E2BF
:100DF000E0E4F9E23DD03CD03BD000914029109195
:100E0000412920914229012B022B047D0FBB109117
:100E1000021420910E1430910F1422533040219F60
:100E2000A001319F500D2091302930913129241794
:100E3000350708F4FD9A0091322910913329209149
:100E40000E1430910F142017310708F4FB9A2091EB
:100E500010143091111440913D2950913E294217B0
:100E6000530708F4F99A0217130708F4F89A08953B
:100E7000002710812D912C3E7CF030911D1417FD20
:100E80003550231714F002E007C030911C1416FDF2
:100E90003B5F32170CF001E0499159916991000FC5
:100EA0003091121414FF365F3617001F000F809127
:100EB0000E1490910F1484179507001F20911014A1
:100EC0003091111442175307001F000F019308952A
:100ED0000091071402FF0FC080910814909109142B
:100EE0004091302950913129EA99C2974817590702
:100EF00010F0EA9A0895EA9808950091071403FF04
:100F00000FC080910A1490910B1440912A2950919E
:100F10002B29EB99C2974817590710F0EB9A0895BF
:100F2000EB98089511E0C0E4D9E2E3E4F9E2EC992A
:100F30003AC00DB30023A9F0E09B089500E20093AE
:100F4000E3050DE20093A60801E00093A30801E089
:100F50000093A5081BD01AD019D000270093A3082E
:100F60000895E09B089500E20093E3050DE20093ED
:100F7000A60801E00093A30801E00093A5080DD0A6
:100F80000CD00BD000270093A3080895099101FD10
:100F900004C002FD04C004FD02C0002700832191AB
:100FA00027DC13950895FE99DCCFFF99DACFE09BFB
:100FB000089500E20093E3050DE20093A60801E026
:100FC0000093A30801E00093A50806D005D004D043
:100FD00000270093A3080895099101FDDECF02FDCB
:100FE000DECF04FFDACFFD9BDACF009119140C702D
:100FF00002950721A1F6D1CF0091432910914429F0
:101000002091452933273EBB0313F09A1313F19A1D
:101010002313F29A0EB30313E69A0895009107146E
:1010200004FF0895EC9B0895009119140C7007219A
:1010300039F0FA990EC0FE990CC0FF990AC00895C4
:10104000FA990895FE990895FF990895FD9920C091
:101050000895009119140C70072109F408951AE0FD
:101060000F9802E00E94600A02E50E94600A012FC8
:101070000E94600A0F9A0F9804E80E94600A0F9A73
:10108000009119140C70009570220FE5802E0895C0
:10109000009119140C70072109F0089519E00F98B8
:1010A00002E00E94600A02E50E94600A012F0E948D
:1010B000600A0F9A0F9804E80E94600A0F9A009144
:1010C00019140C70702A0FE5802E08950D2D0E193D
:1010D000035008F40895D8E2CE2D18811E3F11F078
:1010E000E3940895C3952881C3953881031708F4C4
:1010F0000895C395EC2EE30E27700027E3E8F8E08F
:10110000E20FF01F099407C00FC025C028C02BC0F4
:1011100042C049C04CC011E0311708F40895E89866
:10112000088100FDE89A08951FE1A2E0B4E13117BB
:1011300008F451C049D0C6DA079B089510E80F980B
:1011400002E00E94600A0FE00E94600A012F0E94E4
:10115000600A0F9A94CB18E2A8E0B9E23CC014E010
:10116000ACE1B0E038C014E0AAE4B9E2009144294F
:1011700020E2029F00914329002A00914529000F97
:10118000000F102A1E920E92009004141090051465
:101190001E920E9220C012E0ADEDB9E201E00E9376
:1011A00000E00E9318C01AE0A3E0B1E114C09FDA8A
:1011B0004CDB03E00093A2040E945B0A08ED04BF2D
:1011C00001E00093410008950881C39564D1A3957F
:1011D0001A95D1F70895B59B089500E10093E305B2
:1011E0000DE20093A60801E00093A30801E000933C
:1011F000A50804E40093A70816DB7EF00EEF009329
:10120000A80811DB56F00D910093A8080CDB2EF016
:101210001A95C9F703E00093A40800270093A308D8
:101220000895092D0B7909F4089590FC0BD091FCD9
:1012300014D093FC23D094FC32D097FC3DD0AA2448
:1012400099240895B9E2AEE402E00D93209130298B
:10125000309131293D932D930895B9E2ABE504E037
:101260000D9320912C2930912D293D932D93209180
:101270002E2930912F293D932D930895B9E2A8E6A8
:1012800004E00D93209126292D93209127292D9359
:10129000209128292D93209129292D930895B9E291
:1012A000A5E704E00D932CB32D932DB32D932EB30E
:1012B0002D932FB32D930895002710910F000090C8
:1012C000041410900514A8E0B9E2C3E8D9E2E2E8FA
:1012D000F9E22D913D911694079428F439932993BE
:1012E0000E5F03FD02D01A95A1F700830027259613
:1012F0003D960895E298439481D01FD0519B06D02B
:1013000034D040D0ADD0079907D00895E09981DA64
:10131000A39ABDD0A39808950091071404FF0895DF
:10132000839449F004E6801208950F9802E80E9421
:10133000600A0F9A0895EC98089500910C1400FF2C
:101340000895B5990895E6990895E79B08956394E3
:1013500000910D1460120895CAD977DA03E0009362
:10136000A20448988895489A089540FE089500E39D
:101370000093A00006E00093010606E50093020634
:10138000BB24BBC8B59B089500E10093E3050DE2C3
:101390000093A60801E00093A30801E00093A508CC
:1013A00000E00093A7083FDA2EF10CE00093A808B4
:1013B0003ADA06F105E40093A7082DDADEF0109181
:1013C000A8081123A1F005E00093A40805E4009308
:1013D000A70821DA7EF00091A808D8E2CD2D099364
:1013E000DC2E1A9521F002E00093A408F2CF07E06A
:1013F0000093A40800270093A3080895E09904C06F
:1014000003E00093A2040895E19904C0A99AA19A67
:10141000A098089500911E1410911F142091302956
:10142000309131292017310728F00FB30F7021F0C8
:1014300041FC02C0A99A01C0A998A19A0091201468
:1014400010913F29011710F0A89801C0A89A0EB377
:10145000077011F041FC02C0A09A0895A098089569
:10146000CA9409F00895C0901514009114140B79D2
:10147000902E0895002700938A0A00938B0A01E0BA
:101480000093860A08950091860A00FB0895F2DF12
:10149000FADFF6F708951F93BF93B4E11C91101380
:1014A00003D0BF911F91089506D00C931DE914BF7E
:1014B00013E0109300101091021011FDFCCF08955D
:1014C0000093C4080091C30807FFFCCF0091C40833
:1014D00008954D696C6C73776F6F6420456E676912
:1014E0006E656572696E6720313553204261747490
:1014F0006572792042616C616E6365720D0A46699E
:10150000726D776172652076657273696F6E3A20CD
:10151000312E30300D0A000020000CFFF75E64040D
:1015200080BB7869010F6810D80E1400FF640300B7
:1015300000040100002D68BF32FF7F7F7F7F7F782E
:10154000716B66625E5B585552504E4C4A48464439
:101550004341403E3D3C3A393837363534333231F9
:10156000302F2E2D2C2B2A2A2928272626252423E6
:1015700023222120201F1E1D1D1C1B1B1A19191898
:101580001717161515141313121111100F0F0E0D36
:101590000C0C0B0A0A0908080706050504030201DA
:1015A0000100FFFEFDFCFBFBFAF9F8F7F5F4F3F29E
:1015B000F1EFEEEDEBEAE8E6E4E2FFFFFFFFFFFF0D
:1015C000FFFFFFFFFFFFFFFFFFFFFFFFFFFFFFFF2B
:1015D000FFFFFFFFFFFFFFFFFFFFFFFFFFFFFAF32C
:1015E000EDE7E1DCD6D2CDC8C4C0BCB8B4B1ADAA79
:1015F000A7A4A19E9B999694918F8D8B88868483B6
:10160000817F7D7B7A7877757372716F6E6D6B6A8F
:101610006968666564636261605F5E5D5C5B5A59C0
:101620005857575655545353525150504F4E4E4D94
:101630004C4C4B4A4A49494847474646454544442D
:1016400043434242414140403F3F3F3E3E3D3D3C9F
:101650003C3C3B3B3A3A3A393939383838373737F6
:10166000363636353535343434333333333232323B
:1016700031313131303030302F2F2F2F2E2E2E2E72
:101680002D2D2D2D2D2C2C2C2C2C2B2B2B2B2A2A9D
:101690002A2A2A2A292929292928282828282827BE
:1016A00027272727262626262626262525252525DB
:0A16B00025242424242424242323C9
:00000001FF
